:10000000D8C0FCC0E9C4FAC0F9C09CC4F7C0F6C0AF
:10001000F5C0F4C0F3C0F2C0F1C0F0C0EFC0000002
:1000200000000000000808080808000060600000E8
:10003000003C4030403C003E5149453E0000427F7C
:100040004000004261514946002141454B310018B2
:1000500014127F10002745454539003C4A49493074
:10006000000171090503003649494936000649492E
:10007000291E000036360000007C1211127C007F21
:1000800049494936003E41414122007F4141221CFD
:10009000007F49494941007F09090901003E414962
:1000A000497A007F0808087F0000417F4100002056
:1000B00040413F01007F08142241007F4040404002
:1000C000007F020C027F007F0408107F003E414148
:1000D000413E007F09090906003E4151215E007F33
:1000E000091929460046494949310001017F0101AA
:1000F000003F4040403F001F2040201F003F40384D
:10010000403F002054545478007F4844443800381D
:100110004444442000384444487F00385454541820
:1001200000087E0901020018A4A4A47C001CA0A061
:10013000A07C0000447D4000004080847D00007F62
:10014000102844000000417F4000007C041804781F
:10015000007C0804047800384444443800FC24241B
:1001600024180018242418FC007C08040408004803
:100170005454542000043F444020003C4040207C24
:10018000001C2040201C0000000036000000000081
:100190003800020202020202020202020102040804
:1001A00010202004100801020000040000000000DC
:1001B000A80B11241FBECFE5D2E0DEBFCDBF11E0FA
:1001C000A0E6B0E0EEEBFCE102C005900D92A23299
:1001D000B107D9F721E0A2E2B1E001C01D92A73A30
:1001E000B207E1F710E0C9EDD0E003C02197FE01AE
:1001F0005EDDC83DD107D1F717D45FCD01CF17B869
:10020000369A3699FECF84B195B10895823089F03F
:1002100018F4813051F00895833019F0843009F0DA
:1002200008958CB58F7D8CBD08958AB58F778ABD72
:1002300008958AB58F7DFBCF1F93CF93DF93EAEAB2
:10024000F1E09491E0EAF1E0D491E6E9F1E0C491C3
:10025000CC23B1F0182F992311F0892FD7DFEC2F81
:10026000F0E0EE0FFF1FE457FE4FA591B4918FB75A
:10027000F894EC91111108C0D095DE23DC938FBF68
:10028000DF91CF911F910895DE2BF8CFCF93DF93AD
:10029000E7EAF1E08491EDE9F1E0D491E3E9F1E0FE
:1002A000C491CC2399F08111B1DFEC2FF0E0EE0F77
:1002B000FF1FEA57FE4FA591B491EC91ED2381E029
:1002C00090E009F480E0DF91CF91089580E090E024
:1002D000FACF3FB7F8948091230190912401A09127
:1002E0002501B091260122B708B601FE05C02F3FB7
:1002F00019F00196A11DB11D3FBFBA2FA92F982F4C
:100300008827BC01CD01620F711D811D911D42E046
:10031000660F771F881F991F4A95D1F708958F920E
:100320009F92AF92BF92CF92DF92EF92FF924B01DA
:100330005C01CFDF6B017C01CCDF6C197D098E097C
:100340009F09683E734081059105B0F321E0821A50
:100350009108A108B10888EEC80E83E0D81EE11C00
:10036000F11C81149104A104B10431F7FF90EF90C6
:10037000DF90CF90BF90AF909F908F900895E2E470
:10038000F1E011921186138A81E0EC34F807C9F785
:1003900081E08093420180935601809344018093D1
:1003A00058018093460180935A01809348018093BD
:1003B0005C0180934A0180935E0180934D0180939C
:1003C0004F0180935101809353010895CF92DF92A2
:1003D000EF92FF920F931F93CF93DF932091A4018D
:1003E00021111DC06B017C0110E000E081E024DFE1
:1003F000D0E0C0E0CC16DD0619F000002196FACF5F
:1004000080E01ADF90E080E0C817D90719F00000FB
:100410000196FACF0F5F1F4FE016F1063CF7DF9110
:10042000CF911F910F91FF90EF90DF90CF900895A3
:1004300030E020E090E0AC01022E01C0440F0A94AD
:10044000EAF747FF0CC0C09AC29AC2982F5F3F4F8D
:100450002830310581F7C09AC29AC2980895C09891
:10046000F3CF8130910581F488E9E2DF8CE5E0DFAC
:1004700086EBDEDF8FE5DCDF8FE5DADF86EBD8DFCA
:100480008CE5D6DF88E9D4CF8230910581F480E312
:10049000CFDF8EE3CDDF83EBCBDF8DE5C9DF8DE5ED
:1004A000C7DF83EBC5DF8EE3C3DF80E3ECCF8330B0
:1004B000910581F488E1BCDF88E3BADF84E3B8DF2B
:1004C00084E3B6DF84E3B4DF84E3B2DF88E3B0DF44
:1004D00088E1D9CF892B81F480E0AADF80E0A8DF12
:1004E00080E0A6DF80E0A4DF80E0A2DF80E0A0DF84
:1004F00080E09EDF80E0C7CF0895C298C098C29A7E
:10050000C09A0895C29AC09AC098C2980895CF938D
:10051000DF93C82FD62FF6DF88E78ADF80E088DFF9
:1005200080EB8D0F85DF8C2F82958F70806180DF4F
:100530008C2F8E7081607CDFDF91CF91DECF6830B1
:1005400008F4E5CF0895DEDF88E772DF80E470CF3E
:10055000EF92FF920F931F93CF93DF93EC018C01E7
:10056000060F171F0C171D078CF06C2F80E0E7DFBC
:10057000EADF80E1E82EF12C90E080E072DF81E09C
:10058000E81AF108C9F7B9DF2196ECCFDF91CF91D6
:100590001F910F91FF90EF900895BF92CF92DF923D
:1005A000EF92FF920F931F93CF93DF93B82E8B019F
:1005B000EB0177FD279693E0D595C7959A95E1F7DE
:1005C000C801877099276C2F892BA9F18B2DB7DF74
:1005D000BADFC80168E070E043DBD82F8EE7C82E91
:1005E000D12CE12CF12CD701C6010D2E04C0880FAF
:1005F000991FAA1FBB1F0A94D2F71ADF7EDF6C2F48
:100600006F5F8B2D9CDF9FDF88E08D1BA70196011C
:1006100004C055954795379527958A95D2F7C90116
:1006200007DFDF91CF911F910F91FF90EF90DF9047
:10063000CF90BF9062CF8B2D82DF85DF8EE7F0CF2A
:1006400067E08091A50163DF7EDF80E0F1DE80E07E
:10065000EFDE80ECEDDE80ECEBDE80ECE9DE80ECC2
:10066000E7DE80ECE5DE80EFE3DE80EFE1DE80EFC9
:10067000DFDE80EFDDDE80ECDBDE80ECD9DE80ECDF
:10068000D7DE80ECD5DE80ECD3DE80E0D1DE80E00A
:10069000CFDE33CFAF92BF92CF92DF92EF92FF9235
:1006A0000F931F93CF93DF93D82FE62E6A01F12C7F
:1006B000F601EF0DF11D8081882369F1C0E08032E1
:1006C00051F0C4EDC80FC03130F0CEECC80FC932C4
:1006D00010F0C5ECC80FDF3710F0E394D0E06E2DBA
:1006E0008D2F2DDF30DF8C2F90E066E070E0A7DAF1
:1006F00010E000E0825E9F4F5C01F501E00FF11F0A
:10070000849196DE0F5F1F4F06301105B1F7F5DEBD
:10071000DA5FF394CDCFDF91CF911F910F91FF90CE
:10072000EF90DF90CF90BF90AF900895CF93C82FF8
:10073000E9DE88E77DDE80E07BDE8C2F79DECF91FD
:10074000DCCECF93DF93C0EB8C2FF0DF80E0EEDFC9
:1007500080E1ECDFF8DED0E080E06ADEDF5FD038F9
:10076000D9F7CBDECF5FC83B79F7DF91CF91089502
:10077000B89ABA9A8EEADADF80E0D8DF80E1D6DF75
:1007800080E4D4DF81E8D2DF8FECD0DF81EACEDFF6
:1007900088ECCCDF86EACADF88EAC8DF8FE3C6DFF1
:1007A00083EDC4DF80E0C2DF85EDC0DF80E8BEDF1F
:1007B00089EDBCDF81EFBADF8AEDB8DF82E1B6DF19
:1007C0008BEDB4DF80E4B2DF80E2B0DF82E0AEDF49
:1007D0008DE8ACDF84E1AADF84EAA8DF86EAA6DF41
:1007E0008FEAA4CFEF92FF920F931F93CF93DF93E3
:1007F000CDB7DEB72A970FB6F894DEBF0FBECDBFD8
:10080000F82EE62ECA018E010F5F1F4F2AE0F80175
:1008100011922A95E9F74AE0B8014DD8A8016E2D4A
:100820008F2D38DF2A960FB6F894DEBF0FBECDBFEE
:10083000DF91CF911F910F91FF90EF900895CF938B
:10084000DF93EC011092410110923C0110923B01A8
:10085000109276011092770110927801109279012E
:10086000109298011092990110929A0110929B0196
:10087000109275011092740110926B0110926A012E
:1008800088E090E0909362008093610010922E01C6
:1008900010922D0190932C0180932B0182E090E027
:1008A00090936400809363001092320110923101A2
:1008B00010923401109233011092300110922F01E6
:1008C00010927301109272011092710110927001D6
:1008D00010926D0110926C0181E08093600080E4C1
:1008E00090E09093A6018093A5012BDF44EE50E0A9
:1008F00063E080E1CFDE4BE650E064E080E1CADEF9
:1009000044EE50E065E080E1C5DEAE0164E070E0F9
:1009100085E590E067DF60E273E08EE190E056DD10
:1009200068E572E08EE190E051DD60E971E08EE112
:1009300090E04CDD6CEB72E080E090E0F0DCDF9169
:10094000CF91FFCE1F920F920FB60F9211242F93CB
:100950003F938F939F93AF93BF9380912701909183
:100960002801A0912901B0912A013091220123E0B0
:10097000230F2D3758F50196A11DB11D209322019B
:100980008093270190932801A0932901B0932A0115
:100990008091230190912401A0912501B09126011D
:1009A0000196A11DB11D8093230190932401A09372
:1009B0002501B0932601BF91AF919F918F913F91F7
:1009C0002F910F900FBE0F901F90189526E8230FC0
:1009D0000296A11DB11DD2CF1F920F920FB60F929A
:1009E00011242F933F934F935F936F937F938F9334
:1009F0009F93AF93BF93EF93FF9348DC892B19F438
:100A000081E080934101FF91EF91BF91AF919F9160
:100A10008F917F916F915F914F913F912F910F90A7
:100A20000FBE0F901F90189578948AB582608ABD8A
:100A30008AB581608ABD83B7826083BF83B78160D6
:100A400083BF89B7826089BF80B7826080BF80B76B
:100A5000816080BF329A319A309A379A8CB580641F
:100A60008CBD80E187BB82E085BB8BB780628BBF8A
:100A7000789478EE872E73E0972EA12CB12C78DE37
:100A800060DE47E750E061E080E004DE41E850E0EE
:100A900062E084E0FFDD4DE850E064E080E0FADDF4
:100AA00061E085E534DD4FDD81E090E0DADC90E067
:100AB00080E0D7DC81E090E0D4DC1FDD62E085E5FA
:100AC00026DD41DD90E080E0CCDC82E090E0C9DC16
:100AD00090E080E0C6DC11DD63E085E518DD33DD04
:100AE00090E080E0BEDC90E080E0BBDC81E090E064
:100AF000B8DC90E080E0B5DC81E090E0B2DCFDDCC9
:100B000080E690E09093A6018093A50199DD8FB7D0
:100B1000F894C0902701D0902801E0902901F0902E
:100B20002A018FBFB3DB892B09F0A2C12FB7F8943C
:100B30008091270190912801A0912901B0912A016B
:100B40002FBF8C199D09AE09BF09813D9740A105B2
:100B5000B10544F354DB863B93400CF075C160E073
:100B600090E080E0E3D660E081E090E0DFD64AE903
:100B700050E060E088E08EDDC1E088DB892BE9F39E
:100B8000C11135C5C0E7D0E01C2F8C2F80528831B1
:100B900020F4BE0188E690E000DD1032A9F463E0A5
:100BA00084E6B5DCD0DC90E080E05BDCA6DC64E0D1
:100BB00084E6ADDCC8DC90E080E053DC9EDC64E6DB
:100BC00070E08EE190E002DC60E0812FA0DCBBDC15
:100BD00083E090E046DC90E080E043DC8EDC30DDBA
:100BE00064E170E080E090E09ADB219769F660E0D4
:100BF00080E08DDCA8DC90E080E033DC90E080E0F9
:100C000030DC7BDC47EC50E066E080E043DD43ED28
:100C100050E067E080E03EDD6CED75E080E090E064
:100C20007EDBA6DD8EDD1092A3011092A201109250
:100C3000A101109298011092990110929A011092BC
:100C40009B0181E090E09093660080936500109294
:100C5000A00110929F0110927B0110927A011092D4
:100C600081011092800110928701109286011092EA
:100C70008D0110928C0110929301109292017FDBF2
:100C800081E090E0DCDD22242394312C8091A301CB
:100C900081110EC48091760190917701A091780125
:100CA000B09179010196A11DB11D809376019093B9
:100CB0007701A0937801B093790180919801909188
:100CC0009901A0919A01B0919B010196A11DB11DBE
:100CD0008093980190939901A0939A01B0939B01FE
:100CE00080917401909175010196909375018093A4
:100CF000740185DA9C01255F3140293F310568F494
:100D00002091A5013091A6012F36310534F42F5FD3
:100D10003F4F3093A6012093A5018F5E9240873C00
:100D2000910560F48091A5019091A6018230910512
:100D30002CF001979093A6018093A50180917201F8
:100D400090917301892BD1F45FD5A501940115D63B
:100D5000673E73408105910589F4809170019091FF
:100D600071011816190654F4309273012092720121
:100D70008FE690E090936F0180936E0152E4E52E30
:100D800051E0F52ED0E0C0E08091630090916400C6
:100D90008C179D070CF477C0609170016C0F8091E7
:100DA0006C01880F880F880FCADBCDDB00916A01C8
:100DB00010916B016E01E894C1F8809161009091EF
:100DC0006200801791070CF458C0F701E00FF11F83
:100DD0008081882309F44EC0809163009091640063
:100DE000C817D90731F510D52091650030916600FC
:100DF00047EE442E43E0542E421A530A052C000CB1
:100E000066087708A5019401B8D546165706680606
:100E100079067CF4EAE7F1E090E080E0208131811E
:100E20002130310509F065C401963696853091056B
:100E3000A9F781E090E0C114D10411F082E090E0C4
:100E400010DB0F5F1F4FB9CFC091A401C11108C0C3
:100E500081E08093A4014DEA50E060E080E28BCE17
:100E60001092A40148EB50E060E087E113DC85CEEE
:100E7000C0E083CE90E080E0E3CF3FDB21962AE024
:100E8000E20EF11C81CF4091A1015091A20166E0D8
:100E900070E090E080E0A6DC0091610010916200BB
:100EA00080916A0190916B01081B190BB8E0EB2E41
:100EB000F12CE01AF10AD0E0C0E0CE15DF051CF4F9
:100EC000BFDB2296FACF8091740190917501039750
:100ED0007CF11092750110927401809172019091D1
:100EE0007301892B29F1C0916E01D0916F0160E0EF
:100EF0008C2F0DDB28DB83E090E0B3DA90E080E01C
:100F0000B0DAFBDA2197D0936F01C0936E01CD2B3D
:100F100079F4109273011092720160E080E0F7DAC8
:100F200012DB90E080E09DDA90E080E09ADAE5DA8A
:100F3000809165009091660001976BEF7FEF7FD6FF
:100F4000845A9F4F092E000CAA0BBB0B40917601CF
:100F50005091770160917801709179014817590794
:100F60006A077B078CF1109276011092770110923C
:100F700078011092790180916C0190916D01E0905F
:100F80006300F0906400C0917001D09171012091D4
:100F90006000222309F4EAC12EE030E0201B310B6F
:100FA000821793070CF4DCC110926000B701CE01E8
:100FB000CFDA2196D0937101C0937001B70180916F
:100FC000700190917101C4DA809141018823C9F0C8
:100FD00080913B0190913C01892B99F430923C0126
:100FE00020923B018091A5019091A60108969093D3
:100FF0003E0180933D0188E390E09093400180930F
:101000003F018091980190919901A0919A01B0912E
:101010009B010297A105B1050CF40FC31092980132
:101020001092990110929A0110929B0180913B01BC
:1010300090913C010197D9F4C0913F01D0914001BA
:1010400010913D01BE01812F90913E01A6DA2097BB
:1010500009F095C160E0812F5ADA75DA80E0E8D9AD
:101060004CDA10923C0110923B01109241018091A8
:101070006C0190916D01A3E0880F991FAA95E1F78B
:1010800090933A018093390120914101222309F480
:10109000DFC100913D0110913E01B801681B790B41
:1010A00077FF02C0695F7F4FF3E075956795FA950A
:1010B000E1F7072E000C880B990B35D56B017C01ED
:1010C00060916A0170916B01072E000C880B990BDF
:1010D0002AD59B01AC01C701B6018ED4F1D470931F
:1010E000380160933701C0913F01D0914001BE01AA
:1010F000D7FF02C0695F7F4FE3E075956795EA957A
:10110000E1F7072E000C880B990B0DD56B017C01C4
:101110006091700170917101072E000C880B990B82
:1011200002D59B01AC01C701B60165D4C9D4709347
:10113000360160933501809172019091730101979E
:1011400009F04FC080916E0190916F010817190747
:101150000CF447C00896801791070CF442C02997F9
:101160000CF03FC051D323E630E040E050E005D41E
:10117000AB01BC014F5F5F4F6F4F7F4F8091A1016B
:101180009091A2014E315105610571050CF0FDC031
:10119000C2969093A2018093A10160E971E08EE173
:1011A00090E014D96CE271E08EE190E00FD968EC28
:1011B00070E08EE190E00AD964E670E08EE190E0A4
:1011C00005D9109273011092720160E080916E0156
:1011D0009ED9B9D990E080E044D990E080E041D92F
:1011E0008CD920913D0130913E018091390190913F
:1011F0003A01281739070CF42BC1C0913501D09161
:101200003601D7FD25C1E0906300F0906400EC1634
:10121000FD060CF41DC10091370110913801093011
:10122000110508F015C1CE016AE070E008D58E5BAB
:101230009E4FFC01E00FF11F8081882309F408C153
:10124000C230D10509F0B4C08091330190913401CE
:1012500001969093340180933301809133019091F2
:1012600034018530910521F43092640020926300AE
:1012700040913101509132014430510531F40597CC
:1012800021F4109264001092630083E090E08C1BC4
:101290009D0B6AE070E0D3D44091A1015091A2016E
:1012A000840F951F9093A2018093A10180912F013B
:1012B0009091300101969093300180932F01D0904E
:1012C0007001C09071016C2F6D0D6F5F822F37D947
:1012D0003AD980E0ADD811D964E670E08EE190E0B3
:1012E00075D81092410110923C0110923B0110926E
:1012F0003E0110923D0187E090E090934001809381
:101300003F01CE016AE070E09AD48E5B9E4FFC01F3
:10131000E00FF11F108240916100509162008091B6
:101320006A0190916B010817190709F066C0809156
:101330002D0190912E01FA01EE5BFE4F9A012017CC
:1013400031070CF445C06081611140C062856111B4
:101350003DC0648961113AC0215031093197EFCF06
:10136000019690936D0180936C0128CE1816190692
:1013700024F081E08093600019CE0197F2CF21978D
:10138000D0934001C0933F0172CE4C3351056105AB
:1013900071051CF48C599F4FFCCE4A3551056105EF
:1013A00071051CF48A569F4FF4CE845D9E4FF1CE9A
:1013B000C130D10509F051CF8091310190913201B6
:1013C0000196909332018093310147CFC901C4CF78
:1013D00090932E0180932D019C01201B310B609175
:1013E0006C0170916D01260F371F30936D012093B2
:1013F0006C0190936B0180936A014017510721F5AE
:1014000080916A0190916B0130912B0120912C0108
:10141000FC01EE5BFE4F4817590774F061916111B2
:1014200008C06185611105C06389611102C0019620
:10143000F2CF382F292FFBCF30932B0120932C0193
:101440003093610020936200B7018D2D9C2D80D8D0
:10145000CAE7D1E088819981019709F0E7C00C8142
:101460001D81B8018A819B8198D80F5F1F4F1D8312
:101470000C83083311050CF4D9C067E08A8147D882
:1014800062D880E0D5D739D8198218822A813B8169
:101490008091A5019091A601821793070CF0C6C018
:1014A0004096281739070CF0C1C081E08093A30152
:1014B00090E080E033D2C82FD0E0DC2FCC27D0934F
:1014C000A001C0939F0181E090E028D2C82BD09367
:1014D000A001C0939F016091A1017091A201C61764
:1014E000D7077CF47093A00160939F0181E090E0A6
:1014F0001DD26091A20190E080E018D281E080933B
:101500009C0180919F019091A00190939E018093F6
:101510009D0117D942EE50E061E08BE0BBD843EF6C
:1015200050E062E08BE0B6D842EE50E063E08BE042
:10153000B1D849E051E065E085E2ACD84091A10125
:101540005091A20165E070E08BE490E04BD980916E
:101550009C0181110EC044E051E067E085E19AD81A
:1015600040919D0150919E0167E070E088E590E018
:1015700039D9D0E0C0E0BE0182E390E027D7E296FF
:10158000C83E93E0D907B9F760ED77E080E090E0DE
:10159000C6D680919C01882351F1D3D842EE50E009
:1015A00061E08AE077D840E151E063E08AE072D8F8
:1015B00042EE50E067E08AE06DD840919D01509185
:1015C0009E0165E070E082E390E00CD9CCEBD2E0C4
:1015D000BE018EE190E0FAD6E297C83CD105C1F792
:1015E00010929C016CE87AE080E090E098D6A9D84F
:1015F0008EEA9CD8379885B7877E806185BF85B78E
:10160000806285BF85B7806285BF889585B78F7DED
:1016100085BF85B78F7D85BF379A8FEA87D880E0F1
:1016200090E0892B09F42BCAEBD429CA269688E9C5
:1016300091E08C179D0709F00DCF80912F019091BB
:1016400030010E9751F510927B0110927A011092A1
:1016500081011092800110928701109286011092F0
:101660008D0110928C0110929301109292011092B0
:101670009901109298018091650090916600019601
:1016800080319105DCF49093660080936500809131
:10169000650090916600D3D872D6809170019091C8
:1016A00071018530910569F4809163009091640027
:1016B000029781F481E08093A301E8CA8FE090E073
:1016C000E2CF8630910561F48091630090916400CF
:1016D000019781F38091A3018111ECCFB1D7DACAD0
:1016E0000797C1F78091630090916400892B91F76F
:1016F000E1CF66E070E0A3D2FC01E658FE4F81E046
:1017000090E09183808380916A0190916B019801B0
:10171000281B390B80916C0190916D01820F931FF2
:1017200023E0880F991F2A95E1F70496938382831B
:1017300020917001309171012C0F3D1F2F5F3F4FA1
:1017400043E0220F331F4A95E1F73583248371CBA1
:1017500080916A0190916B0190932E0180932D01ED
:10176000809161009091620090932C0180932B01F5
:1017700008958F929F92AF92BF92CF92DF92EF9295
:10178000FF92CF93DF93EC01688179818A819B81FD
:10179000611571058105910521F464E279ED8BE510
:1017A00097E02DE133EF41E050E0E7D049015A01E5
:1017B00027EA31E440E050E0C7D06B017C012CEE19
:1017C00034EF4FEF5FEFC501B401BED0C60ED71E98
:1017D000E81EF91EF7FE06C081E0C81AD108E1082C
:1017E00080E8F80AC882D982EA82FB82C701B60182
:1017F0009F77DF91CF91FF90EF90DF90CF90BF90D8
:10180000AF909F908F9008958F929F92AF92BF92CA
:10181000CF92DF92EF92FF92609167007091680023
:101820008091690090916A006115710581059105AB
:1018300021F464E279ED8BE597E02DE133EF41E0AF
:1018400050E09BD049015A0127EA31E440E050E0E2
:101850007BD06B017C012CEE34EF4FEF5FEFC501C5
:10186000B40172D0C60ED71EE81EF91EF7FE06C0E0
:1018700081E0C81AD108E10880E8F80AC092670040
:10188000D0926800E0926900F0926A00C701B60148
:101890009F77FF90EF90DF90CF90BF90AF909F9099
:1018A0008F9008956093670070936800809369003B
:1018B00090936A000895BB274A3031F4992322F4AB
:1018C000BDE2909581959F4F01C0BB27FB01552735
:1018D000AA27880F991FAA1FA41710F0A41B83958D
:1018E0005051B9F7A05DAA3308F0A95DA193009704
:1018F00079F7B111B1931192CB0100C0DC01FC0169
:10190000672F71917723E1F7329704C07C916D9333
:1019100070836291AE17BF07C8F30895E199FECFB7
:101920009FBB8EBBE09A99278DB30895262FE1992E
:10193000FECF1CBA9FBB8EBB2DBB0FB6F894E29AAC
:10194000E19A0FBE01960895EE27FF27AA27BB272D
:1019500008C0A20FB31FE41FF51F220F331F441F3F
:10196000551F969587957795679598F37040A9F7D9
:10197000009799F7BD01CF010895052E97FB16F446
:1019800000940FD057FD05D014D007FC02D046F4C8
:1019900008C050954095309521953F4F4F4F5F4F70
:1019A000089590958095709561957F4F8F4F9F4FCB
:1019B0000895A1E21A2EAA1BBB1BFD010DC0AA1F90
:1019C000BB1FEE1FFF1FA217B307E407F50720F0A8
:1019D000A21BB30BE40BF50B661F771F881F991F23
:1019E0001A9469F760957095809590959B01AC016C
:1019F000BD01CF0108955058BB27AA270ED0E5C0DE
:101A0000D6D030F0DBD020F031F49F3F11F41EF43B
:101A1000CBC00EF4E095E7FBC1C0E92FE7D080F31F
:101A2000BA17620773078407950718F071F49EF5DB
:101A3000FFC00EF4E0950B2EBA2FA02D0B01B901BB
:101A400090010C01CA01A0011124FF27591B99F034
:101A5000593F50F4503E68F11A16F040A22F232F40
:101A6000342F4427585FF3CF469537952795A79590
:101A7000F0405395C9F77EF41F16BA0B620B730B37
:101A8000840BBAF09150A1F0FF0FBB1F661F771FA8
:101A9000881FC2F70EC0BA0F621F731F841F48F45D
:101AA000879577956795B795F7959E3F08F0B3CFE3
:101AB0009395880F08F09927EE0F979587950895CD
:101AC00004D06894B111B5C0089598D088F09F579C
:101AD00090F0B92F9927B751A0F0D1F0660F771F7A
:101AE000881F991F1AF0BA95C9F712C0B13081F05A
:101AF0009FD0B1E008959CC0672F782F8827B85FEA
:101B000039F0B93FCCF3869577956795B395D9F7BA
:101B10003EF490958095709561957F4F8F4F9F4FC4
:101B20000895E89409C097FB3EF4909580957095D0
:101B300061957F4F8F4F9F4F9923A9F0F92F96E919
:101B4000BB279395F695879577956795B795F1118E
:101B5000F8CFFAF4BB0F11F460FF1BC06F5F7F4F2B
:101B60008F4F9F4F16C0882311F096E911C077233D
:101B700021F09EE8872F762F05C0662371F096E846
:101B8000862F70E060E02AF09A95660F771F881F15
:101B9000DAF7880F9695879597F9089597F99F67D3
:101BA00080E870E060E008959FEF80EC08950024E5
:101BB0000A941616170618060906089500240A94B2
:101BC00012161306140605060895092E0394000C38
:101BD00011F4882352F0BB0F40F4BF2B11F460FFC7
:101BE00004C06F5F7F4F8F4F9F4F089557FD9058F0
:101BF000440F551F59F05F3F71F04795880F97FBD1
:101C0000991F61F09F3F79F087950895121613068A
:101C10001406551FF2CF4695F1DF08C016161706B9
:101C20001806991FF1CF86957105610508940895EE
:101C3000E894BB2766277727CB0197F908950024FE
:101C4000552704C0080E591F880F991F009729F0C7
:101C500076956795B8F37105B9F7802D952F08959E
:101C600097FB072E16F4009406D077FD08D00BD012
:101C700007FC05D03EF4909581959F4F089570958F
:101C800061957F4F0895AA1BBB1B51E107C0AA1F96
:101C9000BB1FA617B70710F0A61BB70B881F991F0D
:101CA0005A95A9F780959095BC01CD010895EE0F46
:0E1CB000FF1F0590F491E02D0994F894FFCFEA
:101CBE000108000200010001000000204C20452018
:101CCE00562045204C2000532050204120432045D3
:101CDE0000412054205420412043204B00616E646B
:101CEE0068206A61636B736F6E002D484947482008
:101CFE0053434F52452052455345542D002D2D2010
:101D0E004D555445202D2D002D2D20534F554E440D
:101D1E00204F4E202D2D00696E7370697265642000
:101D2E006268002F6562626F67676C65732E636F02
:101D3E006D002D2D2D2D2D2D2D2D2D2D2D2D2D2DB2
:101D4E002D2D00472041204D204520204F2056208C
:101D5E0045205200484947482053434F52453A00C8
:101D6E00204E455720484947482053434F5245205F
:021D7E00000063
:00000001FF
